:1000000089C300000C94B72FBDC30000BBC3000020
:10001000B9C30000B7C30000B5C30000B3C30000FC
:10002000B1C30000AFC300000C94ED2D0C94D52E8D
:100030000C94A22DA7C30000A5C30000A3C3000019
:10004000A1C300009FC300009DC300009BC300002C
:1000500099C300000C94C92D95C3000093C3000000
:1000600091C300008FC300008DC300008BC300004C
:1000700089C3000087C3000085C3000083C300005C
:1000800081C300007FC300007DC300007BC300006C
:1000900079C3000077C3000075C3000073C300007C
:1000A00071C300006FC300006DC3000005010902A9
:1000B000A10185020901A1000509190129081500FE
:1000C0002501950875018102050109300931158165
:1000D000257F95027508810609381581257F9501D0
:1000E00075088106050C0A38021581257F95017572
:1000F000088106C0C005010980A101850319012AF4
:10010000B700150126B700950175108100C0050CD8
:100110000901A101850419012AA002150126A002E6
:10012000950175108100C00660FF0961A101096297
:10013000150026FF00952075088102096315002629
:10014000FF00952075089102C005010906A101056F
:100150000719E029E7150025019508750181029529
:1001600001750881010507190029FF150026FF0008
:100170009506750881000508190129051500250156
:10018000950575019102950175039101C00000006C
:10019000000000000000000000000000000000005F
:1001A000000000000000000000000000000000004F
:1001B000007E0F00D4FFFFFFC700000078000000A2
:1001C00000000000002A2B280000000000000000B2
:1001D000000000000000000029000000002C1E3478
:1001E00020212224342627252E362D3738271E1F7E
:1001F000202122232425263333362E37381F0405A9
:10020000060708090A0B0C0D0E0F10111213141516
:10021000161718191A1B1C1D2F3130232D350405F4
:10022000060708090A0B0C0D0E0F101112131415F6
:10023000161718191A1B1C1D2F3130354C09025B7B
:1002400000030100A0FA09040000010301010009F4
:100250002111010001224400070581030800010962
:100260000401000203000000092111010001222203
:100270000007058203200001070503032000010990
:100280000402000103000000092111010001227B8A
:10029000000705840320000112010002000000088D
:1002A00010CB56310003010203011C0376006900E4
:1002B00061006C003A0066003600340063003200D2
:1002C00062003300630000001E034E0079007100DD
:1002D000750069007300740020005200650076000C
:1002E0002E002000330000000E034B006500650067
:1002F000620069006F0000000403090435001E005D
:100300001F002000210022002B0014001A0008000A
:1003100015001700290004001600070009000A0054
:10032000E1001D001B000600190005002552E00039
:10033000E200E30023522C002300240025002600C5
:1003400027002A001C0018000C00120013004C00AB
:100350000B000D000E000F003300340011001000E0
:1003600036003700380028002C002452500051007D
:1003700052004F0035001E001F0020002100220007
:100380002B0014001A00090013000A0029000400C1
:100390001500160017000700E1001D001B000600F5
:1003A000190005002552E000E200E30023522C0072
:1003B000230024002500260027002A000D000F003E
:1003C00018001C0033004C000B00110008000C004A
:1003D000120034000E0010003600370038002800EC
:1003E0002C0024525000510052004F0035001E00D6
:1003F0001F002000210022002B00340036003700AF
:1004000013001C00290004001200080018000C0052
:10041000E100330014000D000E001B002552E00027
:10042000E200E30023522C002300240025002600D4
:1004300027002A0009000A00060015000F004C00E2
:1004400007000B001700110016003800050010000F
:100450001A0019001D0028002C00245250005100E1
:1004600052004F0035021E021F022002210222020A
:1004700035021E021F022002210222024C003A0015
:100480003B003C003D003E0005784000410042003A
:1004900043004400010001000100010001000100CF
:1004A000230224022502260227022A002302240214
:1004B0002502260227024C003F002D022E022F02A9
:1004C000300231024500320264024A004D00010050
:1004D00001000100AB00AA00A900AE0035001E001B
:1004E0001F0020002100220035001E001F002000F8
:1004F000210022004C003A003B003C003D003E0041
:10050000010040004100420043004400010001009E
:100510000100010001000100230024002500260045
:1005200027002A00230024002500260027004C0075
:100530003F002D002E002F0030003100450032001A
:1005400064004B004E00010001000100AB00AA0056
:10055000A900AE003A003B003C003D003E003F00D9
:100560000100007C4278437846784578010001001C
:100570000100807481741570010001000100010008
:100580000100010001000100010001000100010063
:10059000400041004200430044004500487847784D
:1005A0004A78497801004C0014704052415242523E
:1005B0000100010001000100010001000100010033
:1005C000010001000100010001000100FD377A581F
:1005D0005A000004E6D6B4460200210116000000CD
:1005E000742FE5A3E003B201085D003D888986D33E
:1005F000DC0AE842C3249258425AFA4B42162C5F56
:10060000542BA3199BCDF09E3ED52B7388208A27AF
:1006100002C28C6C91863337C68276CB812B45B073
:100620004557660343EA9B6B19E8B1AAA5E31F2C63
:1006300065784B4034F572DD554C0E88976FFB9210
:100640000FB4A5F05BB19A2B1D54928E8272F648BE
:10065000E7B4799F489284ADB1C6FC79939A8D1C1A
:1006600035FF1B43F6C6C36EBA331667230739003E
:1006700080DCF0C90C81E00A7D63DD01534C5B95A1
:10068000B69BDD20F18041788D582E31A49DE6E4A3
:1006900022C3AEFD3C42DB72E04C0613E4B985296F
:1006A000FF5AE82552FB2F1DAE76F50CE6A9333E26
:1006B000C260D50808F250A7490CB73F7F5CCCBB9D
:1006C0008B1564DEBF6F0059C9DDAAEC69D00951F2
:1006D000F1D362269E135492CC3819E51A9CEAD3C2
:1006E00022865F6703DF3AED5FB76A10E5AD968D4E
:1006F0004D7F0000B6C38E336581AEE60001A402D3
:10070000B3070000B4239031B1C467FB02000000BE
:100710000004595A11241FBECFEFDAE0DEBFCDBF6F
:1007200004B603FE18C08091F2039091F303A091E8
:10073000F403B091F5038730904BA740B04B59F4C8
:100740001092F2031092F3031092F4031092F50347
:10075000E0E0F8E3099511E0A0E0B1E0EEEEF4E6A8
:1007600002C005900D92A43CB107D9F723E0A4EC98
:10077000B1E001C01D92A23FB207E1F70E949926A5
:100780000C9402323DCC9C019A9581159F4118F53D
:10079000F32FF270EE27832F8170732F747066270A
:1007A000532F5870442734FF0CC08295807FEF2B65
:1007B00009F08062672B09F08064452B69F080683E
:1007C0000895EF2B09F08260672B09F08460452BB8
:1007D00019F08860089580E00895CF93DF93EB01CE
:1007E000D2DFFE010995DF91CF910895982F929560
:1007F0009F7024E0911102C020E0982F892F8695E8
:100800008695811511F02E5F982F892F8695820F7E
:1008100008958093A70308958093A803089521E085
:1008200030E001C0220F8A95EAF78091A803822B5D
:10083000F3CF21E030E0A90102C0440F551F8A9593
:10084000E2F7CA0180959091A8038923E5CF292F6B
:100850009A3090F5863080F590E036E0239F800D49
:10086000911D1124282F277041E001C0440F2A95C3
:10087000EAF723E0969587952A95E1F7FC01EE0FBC
:10088000FF1FE80FF91FE859FD4F20E030E070E04E
:100890005191DF01CB01022E02C0969587950A94F3
:1008A000E2F7817081958527842385278E932F5FBA
:1008B0003F4F2330310561F70895292F9A3078F59D
:1008C000863068F590E036E0239F800D911D11245D
:1008D000682F677023E0969587952A95E1F7FC01CC
:1008E000EE0FFF1FE80FF91FE859FD4F40E050E001
:1008F00080E0219130E0062E02C0369527950A94BB
:10090000E2F721703327042E01C0220F0A94EAF780
:10091000822B4F5F5F4F4330510559F7089580E0B8
:1009200008959091A80321E030E0F90101C0EE0F95
:100930008A95EAF7D90102C0AA0FBB1F6A95E2F7B0
:10094000EA2B01C0220F4A95EAF7892F8E23E8137C
:1009500003C0892F822B60CF2095822F8923FBCF64
:100960008091B0039091AF03981301C008958F5FF9
:100970008770FACF9091AA03809589238093AA0368
:10098000282F2770211110C0891771F09091F10361
:1009900092FF0AC08695869586954BDF1092AA0332
:1009A0001092AC031092AB0308959091A503982B7D
:1009B0009093A5030895982F90958091A50389237E
:1009C0008093A50308958091A403811531F01092BE
:1009D000A4031092AE031092AD030895803E9105DA
:1009E000D9F1C8F48133910509F482C048F4893201
:1009F000910509F472C08A32910509F480C0089506
:100A000089339105E9F082389105D1F0853391055C
:100A100009F45EC00895843E9105D9F148F4823E00
:100A2000910539F1833E910549F181EE90E00895F9
:100A3000863E9105C9F1873E910509F43EC00895AF
:100A40002091F0032370211164C02091F10323FF52
:100A500014C089E290E008952091F00320FD45C084
:100A60003091F10330FF09C024FD24C083EE90E0F3
:100A700008952091F00322FDF7CF08952091F0030F
:100A800022FD44C03091F10330FD43C024FFF5CF77
:100A900011C02091F10321FFF0CF8091F00384FD7C
:100AA00009C087EE90E008952091F00323FFE5CF81
:100AB00024FFF7CF80E090E008952091F00323FD1C
:100AC0002BC03091F10331FFE1CF84EE90E0089527
:100AD0002091F00325FFD1CFBCCF2091F00325FD5D
:100AE0001EC02091F10323FFC8CF89E390E0089551
:100AF0002091F00326FFC1CF8AE290E00895209173
:100B0000F00326FFBACF81E390E0089582EE90E0F3
:100B1000089580EE90E0089586EE90E0089585E3D4
:100B200090E008959091F00392FF10C041E0282FCB
:100B30002471243009F040E031E0282F287128305A
:100B400009F030E0431711F02CE0822793FF10C02A
:100B500041E0282F2471243109F040E031E0282FB2
:100B60002871283109F030E0431711F02CE082277A
:100B70003091F10330FF10C051E0282F2171213056
:100B800009F050E041E0282F2871283009F040E0BA
:100B9000541711F029E0822731FF10C041E0282FBF
:100BA0002171213109F040E031E0282F28712831EE
:100BB00009F030E0431711F029E0822794FD877E89
:100BC00008951F93CF93DF9309DFEC01811522E590
:100BD000920708F052C0811540E5940708F0CDC097
:100BE000803E910520F58D3C910508F0A1C0883A22
:100BF000910570F4853A910508F097C08130910510
:100C0000B9F10497813A910598F1C0E0D0E030C085
:100C1000885A91094B97C8F7C85AD0E0CC0FDD1F0E
:100C2000C95ADE4F0990D881C02DD46421C08115E6
:100C300050E49507B0F4C11580E2D80708F0B3C0BE
:100C4000C83ED105A8F0CE019A9581159F41E8F6DE
:100C50008D2F68DF182FCE019927C0DEEC01D12B34
:100C600007C09927BBDECC27DF70C82BD92BD06AF1
:100C7000CE01DF91CF911F910895803842E594070E
:100C8000C8F5803652E5950708F05BC0C03482E5B0
:100C9000D807D0F4C03292E5D90708F04BC08C2FAA
:100CA0008695869520E2829FC0011124C37021E0C1
:100CB00030E0A90102C0440F551FCA95E2F7EA01CE
:100CC000C82BD92BDD68D4CF8C2F8695869587705D
:100CD00050E2859FC0011124C37021E030E0A901DA
:100CE00002C0440F551FCA95E2F7EA01C82BD92B61
:100CF000DC68BECF803C52E5950758F48F71C03A4E
:100D0000D245A0F590E0982F8827EC01C46FD06AF7
:100D1000AFCF805C9245809708F077CFDC2FCC274F
:100D2000CC27DF71C06FD06AA3CFA497D064A0CFC7
:100D3000D0659ECFCF71D0E0DC2FCC27C16FD06AB9
:100D400097CF86958695877020E2829FC0011124F7
:100D5000C37021E030E0A90102C0440F551FCA95BD
:100D6000E2F7EA01C82BD92BDA6882CFDBDEC82F85
:100D7000D0E0DC2FCC27D0627BCF8F71D3DE93E025
:100D8000CC0FDD1F9A95E1F7CC27DF70282F30E0DC
:100D900084FF05C050E1859F900111243327C22BA9
:100DA000D32BD06965CF8D2F8F71BCDE182FCE016C
:100DB000992714DEEC01D12BDECF80E00895F89462
:100DC000E82FE295EF70F0E041A18F7021E030E074
:100DD000B90102C0660F771F8A95E2F7CB01962F03
:100DE0009095942391A392A1892B82A3789408953E
:100DF000A0E0B0E0EEEFF6E00C94D030883080F563
:100E000081112FC0909180009F7790938000209156
:100E1000860030918700A82FB0E00E94623127E061
:100E200030E040E050E00E94333169017A01809166
:100E30008600909187006CE070E00E940C31621790
:100E4000730798F0C90169E070E00E940C3170935B
:100E5000890060938800CDB7DEB7E8E00C94EC30F1
:100E600087E0909180009068D0CF8091860090912B
:100E700087000091860010918700209186003091B4
:100E80008700C6E0D0E0BE010E940C31C60ED71E1E
:100E9000E11CF11C85E0CC0CDD1CEE1CFF1C8A95CE
:100EA000D1F7C801BE010E940C3140E050E0260F8E
:100EB000371F411D511DC701B6010E943331690121
:100EC0007A01E0918600F0918700CA01B9010E9481
:100ED000FD309B01AC01DF010E9471319B01AC012F
:100EE000C701B6010E94FD302FE096958795779552
:100EF00067952A95D1F720918600309187002617B3
:100F000037071806190608F0A2CF60918600709185
:100F100087009DCF883008F087E0209193022770EA
:100F2000982F990F990F990F922B9093930221E08C
:100F3000983008F420E09091930220FB90F9909370
:100F4000930256CF81152CE7920741F4209133028A
:100F500030913402232B11F480E090E00895EDE10C
:100F6000F3E080E090E067E575E24AE755E22CEEB9
:100F700035E2778366835187408733872287978757
:100F80008687019670968830910599F70895FC013F
:100F90008481862381110AC082818115B9F068237A
:100FA000908593FF05C081E061110FC080E0089536
:100FB000282F22952F708F70282B962F92959F7037
:100FC0006F70962B81E02913F1CF089581E0089589
:100FD0000F931F93CF9301E010E0082E01C0000F84
:100FE0000A94EAF7C091A3039C2F9023911115C096
:100FF0009091AA03969596959695891306C010929E
:10100000AA031092AC031092AB0309DCC027C09373
:10101000A303CF911F910F9108950BDCF7CF282FD9
:1010200035EB2303C001112497FF04C080589109B8
:10103000892F089580589F4FFBCF8091820280FDB9
:1010400014C081FD14C082FD16C0809181028115FB
:1010500081F08E3180F420E5829FC00111246EE181
:1010600070E00E942031862F089584E1089588E27F
:10107000089588E0089580E508958091820280FDBA
:1010800017C081FD17C082FD19C0809180028115B3
:1010900099F0883298F428E0829FC001112468E218
:1010A00070E00E9420316115710551F0862F08957E
:1010B00062E0FCCF64E0FACF61E0F8CF68E0F6CF01
:1010C00081E00895FA01309709F00995089580911B
:1010D0005202811569F0E0915E02F0915F02309753
:1010E00039F00190F081E02D309711F009950895C5
:1010F00080E00895A3E0B0E0E0E8F8E00C94D6309A
:101100009C018091F4019091F50182179307B1F051
:101110003093F5012093F401E0915E02F0915F02BB
:10112000309761F00084F185E02D309739F083E04D
:1011300089833B832A83CE01019609952396E2E0B9
:101140000C94F230A3E0B0E0E8EAF8E00C94D6307A
:101150009C018091F2019091F30182179307B1F005
:101160003093F3012093F201E0915E02F0915F026F
:10117000309761F00084F185E02D309739F084E0FC
:1011800089833B832A83CE01019609952396E2E069
:101190000C94F230A8ECB1E0EFEF90E02D918217C3
:1011A00051F0EF3F19F4211101C0E92F9F5F9630F4
:1011B000A9F7EF3F09F408950E2E000CFF0BEA5338
:1011C000FE4F82830895E8ECF1E09191891302C00B
:1011D000DF011E9291E0EE3CF907B9F70895809186
:1011E000010108952FB7F8948091EE019091EF01DD
:1011F000A091F001B091F1012FBF0895962F209199
:10120000F10322FF0EC0682F660F660F660F692B71
:101210006093AA0304DBE6DF9093AC038093AB03F7
:101220000895FDCA9091A403292F2823211559F070
:10123000809589238093A403811531F0D3DF8093B7
:10124000AD039093AE03089580E090E0F8CFCADF3D
:101250002091850230918602232B211521F0809365
:101260002202909323022091870230918802232B3F
:10127000211521F08093200290932102E0915E02DB
:10128000F0915F02309759F00680F781E02D30979A
:1012900031F082E08093830283E892E0099508951B
:1012A000611509F441C0E3E3E80FE33148F4F0E0ED
:1012B000EC5FFD4C0C945531C0DE81958093860225
:1012C000C6CFBBDEFBCFB9DE819580938502F8CF18
:1012D000B4DEFBCFD2DE80938702F2CFCEDE8195E3
:1012E000FACFCBDE819580938802EACFC6DEFBCFB2
:1012F000815D990B21E030E001C0220F8A95EAF769
:1013000080918402822B80938402DACF80918202C2
:10131000816080938202D4CF809182028260F9CF73
:10132000809182028460F5CF409185028D3C59F412
:101330008091860287FF0DC010928602411559F4F4
:101340001092810208C08E3C81F4809186021816AA
:101350009CF3411581F08091870290918802892B3E
:101360008111AECF10928002ABCF8F3C41F447FF8A
:10137000F0CF10928502809186028115E0CF803DEA
:1013800019F41416B4F3E5CF90918702893D29F43E
:101390001916FCF610928702DCCF8A3D19F497FFEC
:1013A000D8CFF8CF909188028B3D29F497FFD1CF09
:1013B00010928802CECF8C3D19F41916CCF3C9CF08
:1013C0009FE2980F983090F4815D990B21E030E016
:1013D000B90102C0660F771F8A95E2F7CB018095AD
:1013E00090918402892380938402B3CF8D3D31F4A0
:1013F000809182028E7F80938202ABCF8E3D21F45A
:10140000809182028D7FF7CF8F3D09F0A2CF80912E
:1014100082028B7FF0CF2FB7F8946091EE0170912C
:10142000EF018091F0019091F1012FBF08950F938A
:101430001F9380915202811521F0EDDF1F910F91D2
:101440000895E9DF0091540210915502209156024F
:1014500030915702600F711F821F931FEFCFCF9201
:10146000DF92EF92FF92CF93DF93D82FC92FC090D6
:101470001703D0901803E0901903F0901A03CBDF04
:101480006C197D098E099F09643F714081059105A2
:1014900010F1C1DF6B017C0182E390E0A0E0B0E0DD
:1014A000C0921C02D0921D02E0921E02F0921F0216
:1014B0008093180290931902A0931A02B0931B0212
:1014C000D0931503C0931603DF91CF91FF90EF9057
:1014D000DF90CF90089584EF91E0A0E0B0E0E0CFFE
:1014E0000895FC019B018091E4019091E50186172C
:1014F000970740F0672B29F48091E8008E7780935E
:10150000E800C90140E0009741F4411106C0809114
:10151000E80082FF2FC080E0089520913502211558
:10152000A9F12530A9F12091E80023FD2DC02091DB
:10153000E80022FDECCF2091E80020FFE4CF3091BD
:10154000F3002091F200009719F02830310558F08F
:1015500041E02830310509F040E02091E8002E7785
:101560002093E800D0CF41914093F10001972F5F85
:101570003F4FE9CF80913502811541F0853041F030
:101580008091E80083FFC3CF81E0089582E0089551
:1015900083E008958091DE0187FF13C08091E80009
:1015A00082FF06C08091E8008B778093E800089561
:1015B000809135028111F2CF089580913502811515
:1015C000D9F38091E80080FFF8CF8091E8008E7712
:1015D000ECCF2091E4003091E50095E6A90120913F
:1015E000EC00822F817020FF06C08091E80080FF10
:1015F00006C080E008952091E80022FD1AC0809185
:101600003502811589F0853089F08091EB0085FDE8
:101610000FC02091E4003091E50042175307F9F222
:101620009A95E1F684E0089582E0089583E00895B4
:1016300081E00895E8EDF0E080818E7F8083109254
:10164000E2001092DA001092E100A0EEB0E08C917E
:1016500081608C9380818F77808319BCA7EDB0E087
:101660008C918E7F8C9380818F7E80831092DD01A0
:101670000895E0915E02F0915F02309739F00284A4
:10168000F385E02D309711F060E209950895FC0193
:10169000AC014B5F5F4F8FEF61E39191892728E0A9
:1016A00030E0982F990F87FF09C0892F8627215096
:1016B0003040B9F7E417F50781F70895892FF7CF80
:1016C000982F9093E900891771F07091EC002091A8
:1016D000ED005091F00021FD09C09F5F973089F720
:1016E0008093E9000895762F242F50E03091EB008D
:1016F0003E7F3093EB003091ED003D7F3093ED0065
:101700003091EB0031603093EB007093EC0020934C
:10171000ED005093F0002091EE0027FDDECF0895FC
:10172000A0E0B0E0E6E9FBE00C94D030C8EDD0E0FA
:1017300088818F7E8883E7EDF0E0808181608083FF
:1017400084E082BF81E08093DD0188818E7F888381
:1017500002EE10E0F80110821092DA0081EEC82E3D
:10176000D12CF601108288818F77888388818068E8
:10177000888388818F7D888319BC109235021092EE
:10178000DC0110920C021092DB0190EEE92EF12C9C
:10179000F70180818B7F808388818160888342E02C
:1017A00060E080E08DDFF60180818E7F8083F8012C
:1017B000808181608083808188608083F70180815F
:1017C0008E7F8083888180618883CDB7DEB7E8E033
:1017D0000C94EC30E091B0039091AF0327E0E91353
:1017E00002C080E00895AE2FB0E02E9FF0011124DA
:1017F000EF54FC4F3181361306C03081381303C0DB
:101800003581341304C0FD013196E770E8CF81E0E3
:10181000089581E08093E00080E28093D8001092E8
:10182000C9008FE19EE40197F1F700C0000087E056
:1018300090EBDC018093F2039093F303A093F40305
:10184000B093F50388E19CE00FB6F894A8958093D7
:1018500060000FBE90936000FFCF0F931F93CF9354
:10186000DF938B01EA0190913502943051F580931A
:10187000E9008FEF9091E80095FD06C095ED9A95EF
:10188000F1F700008A95B1F78091E80085FF19C053
:10189000A0DE811111C08091E80085FD06C0809115
:1018A000E8008E778093E800F3CFF80181918F01F3
:1018B0008093F100219779F78091E8008E778093EB
:1018C000E800DF91CF911F910F910895792F603239
:1018D00029F440E250E0682F82E0BFCF0895CF9313
:1018E000DF93D82FC92F48E050E0682F792F81E08F
:1018F000B4DF88E0ED2FFC2FA6EEB1E001900D9251
:101900008A95E1F7DF91CF910895BC0146E050E060
:1019100084E0A3CFBC0143E050E084E09ECFA0E090
:10192000B0E0E5E9FCE00C94CE30F82EE92EB62EBE
:10193000A72E8A018091D8019AE0C92ED12C8A3035
:1019400018F0CC24C394D12CC1E0D0E06B2D7A2DBB
:101950008F2D9E2DF8010995811116C02196CC1668
:10196000DD0694F0CC9FC001CD9F900D900D112409
:1019700020E030E045E34A95F1F700002F5F3F4F4C
:1019800028173907B9F7E2CFCDB7DEB7EAE00C94F4
:10199000EA30CF93DF93C1E0D0E001C0CC0F8A954D
:1019A000EAF76C2F83E090E00E94CD318C2F0E94EB
:1019B0000904DF91CF910895FC01608186E090E0F9
:1019C0000C94CD318091930280FD11C08160809391
:1019D0009302813019F489E08093930283E992E0C5
:1019E000EBDF8091930286958695869501CA0895CE
:1019F0001F93CF93DF93962F122F632F8630D8F447
:101A00009A30C8F44630B8F4C42FD0E0CC0FDD1FB4
:101A10002CE0929FC00DD11D112498E7899FC00D25
:101A2000D11D1124CE0189960E94CD31612FCE01A6
:101A30008A960E94CD31DF91CF911F9108959091A8
:101A4000F10392FB222720F9281779F080FB92F905
:101A50009093F1036091F0037091F10384E090E0C2
:101A60000E94E73182E00C94BA040895CF93DF938B
:101A7000C091A5038091A903C82B8091A40381156F
:101A8000F1F0B0DB2091AD033091AE03821B930BDC
:101A90008838934110F00E94E304D091A40320E021
:101AA00088EC91E0FC013081019631112F5F31E02B
:101AB0008E3C9307B9F721110E94E304CD2B80914E
:101AC000990280958C2390919802892B8093C6016E
:101AD00048E050E060E672E086EC91E00E948431DC
:101AE000892BB9F088E0E6ECF1E0A0E6B2E00190E5
:101AF0000D928A95E1F7E0915E02F0915F023097D6
:101B000041F00280F381E02D309719F086EC91E0EE
:101B10000995DF91CF910895CF931092A503C6E068
:101B2000E8ECF1E0DF018C2F1D928A95E9F780E067
:101B300090E0E0DA80E090E005DB1092A90396DF08
:101B4000E3E8F2E0DF011D92CA95E9F71092810205
:101B500010928002109282027ADBCF910895DCDF2E
:101B60002FEF84E39CE0215080409040E1F700C0DB
:101B7000000088E19CE00FB6F894A895809360007F
:101B80000FBE90936000FFCFAAE2B0E0EAECFDE068
:101B90000C94D5308EED91E0FC0101962091F1007E
:101BA000208321E0863E9207B9F78091DF018930DA
:101BB00009F457C0C8F4823009F4B2C0833009F484
:101BC00082C0813081F18091E80083FFE6C080917E
:101BD000DE019091DF019A3008F0DFC0E92FF0E0DC
:101BE000E95EFD4C0C9455318A3009F489C08B3084
:101BF00051F78091DE01813231F78091E2019091BD
:101C0000E301892B01F78091E800877F8093E8004A
:101C1000C1DC81E09091E001911101C080E08093EE
:101C200002017ADFD0CF8091DE01813A61F68091A6
:101C3000E800877F8093E8008091E2019091E301C2
:101C4000892B59F060E080E090E070E04ADC809100
:101C5000E8008B778093E800B6CF68E086EE91E0ED
:101C6000F4CF8091DE01813209F0ADCF8091E201A5
:101C70009091E3018D7F892B09F0A5CF8091E80039
:101C8000877F8093E8008091E80082FF17C09091E1
:101C9000F3008091F200029731F48091F1008130DD
:101CA00011F0863021F48091F10080930101809140
:101CB000E8008B778093E8006DDC85CF809135025A
:101CC0008111E1CF80CF8091DE01813A09F07BCF95
:101CD0008091E2019091E301892B09F074CF80910A
:101CE000E800877F8093E8008091E80080FFFCCFC8
:101CF000809102018093F1008091E8008E77DACF25
:101D00008091DE01813209F05ECF8091E800877F0B
:101D10008093E8003FDC8091E1018093000153CF84
:101D20008091DE01813A09F04ECF8091E800877FF3
:101D30008093E8008091E80080FFFCCF8091000153
:101D4000D9CF803889F0823841F58091E2018F70D7
:101D5000873018F58093E9008091EB0085FB882798
:101D600080F91092E90006C080910C02880F9091D2
:101D7000DB01892B9091E800977F9093E800809396
:101D8000F1001092F1008091E8008E7723C081115C
:101D900016C08091E001813009F18091E80083FF55
:101DA0000AC08091E800877F8093E8008091EB0073
:101DB00080628093EB00AA96E3E00C94F1308230CD
:101DC00061F78091E001811581F01092E900809126
:101DD000E800877F8093E800DDDBDFCF81E0933090
:101DE00009F080E080930C02F0CF8091E2018F70C7
:101DF0002FEF280F263088F68093E9002091EB0022
:101E000020FFE3CF933031F48091EB008062809328
:101E1000EB00DBCF9091EB0090619093EB0021E021
:101E200030E0A90102C0440F551F8A95E2F74093A4
:101E3000EA001092EA008091EB008860E8CF8111FF
:101E4000ACCF1091E0011F778091E3008078812B67
:101E50008093E3008091E800877F8093E8009ADB1D
:101E60008091E80080FFFCCF8091E3008068809340
:101E7000E30083E0111101C082E0809335028DCF31
:101E80008058823008F089CF8091E0019091E10183
:101E90008C3D53E0950791F583E08A838AE289833C
:101EA0004FB7F894DE01139620E03EE051E2E32FB5
:101EB000F0E050935700849120FF03C082958F700B
:101EC0003F5F8F708A30C0F0895C90E08D939D9366
:101ED0002F5F243161F74FBF8091E800877F8093A7
:101EE000E8006AE270E0CE010196FBDA8091E8003A
:101EF0008B778093E80051CF805DE7CF292F332780
:101F00002330310509F44EC078F52130310509F44C
:101F100088C08BE590E0EDE3F2E02230310509F076
:101F20003CCF2091E800277F2093E8002091E40136
:101F30003091E5018217930708F49C0140E02115D8
:101F4000310509F073C0411171C08091E80082FD34
:101F5000CDCF80913502811549F2853039F28091DB
:101F6000E80083FFF2CFC2CF8091E2019091E301BC
:101F70002132310509F446C02232310509F00DCF76
:101F80008330910508F009CFFC01EE0FFF1FE25CE2
:101F9000FE4F0190F081E02D855C9E4FDC018C911D
:101FA00090E010C09C013327823021F123303105AD
:101FB00068F4232BB9F4E8EFF2E0E4918E2F90E07F
:101FC000E8EFF2E0009709F4E8CEABCF233031051B
:101FD00009F0E3CEEAEAF2E0E4918E2F90E0EAEA3B
:101FE000F2E0F0CFE8EEF2E0E4918E2F90E0E8EE40
:101FF000F2E0E8CFE8ECF2E0E4918E2F90E0E8EC3C
:10200000F2E0E0CF8330910508F0C7CEFC01EE0F7F
:10201000FF1FEC5BFE4F0190F081E02D89E090E026
:1020200080CF82E190E0E8E9F2E07BCF8091350259
:10203000811509F45BCF853009F458CF8091E80011
:1020400083FD54CF8091E80082FD7FCF8091E8002E
:1020500080FF75CF9091F3008091F200211531053A
:1020600019F08830910550F041E0089709F040E000
:102070008091E8008E778093E80061CF449140938F
:10208000F1003196215031090196E8CF803809F0EE
:1020900084CE8091E800877F8093E8008091DC0106
:1020A0008093F10070CE811178CE1091E001123052
:1020B00008F073CE8091E800877F8093E80010934A
:1020C000DC0168DA1115D9F084E08093350242E032
:1020D00061EC81E0F5DA42E261EC84E0F1DA42E2BF
:1020E00061EC82E0EDDA42E260EC83E0E9DA8091D3
:1020F0003502843051F482E0809303014ECE80910A
:10210000E30087FDE1CF81E0E0CF81E0F5CFCF9321
:10211000C82F8115A9F08238A9F40E94670881FDB3
:102120000FC089E337D8A2DC2FEF37EE83E02150D0
:1021300030408040E1F700C0000089E344D896DCDD
:10214000CF910895833891F40E94670880FDF8CFFD
:1021500083E520D88BDC9FEF21EE34E091502040C6
:102160003040E1F700C0000083E5E8CF843891F407
:102170000E94670882FDE4CF87E40CD877DC8FEFFC
:1021800091EE24E0815090402040E1F700C0000033
:1021900087E4D4CF8CEF8C0F813A70F4E8ECF1E057
:1021A0008EEC91E02191C217B1F18E179F07D1F704
:1021B0008C2F0E94CA08C3CF80E28C0F883048F46D
:1021C000C77081E001C0880FCA95EAF70E94D50464
:1021D000B6CF8BE58C0F833038F42C2F2452330B81
:1021E000C9010E947A08ACCFE8E5EC0FEB3150F45E
:1021F000F0E0EE0FFF1FE357FE4F808191810E94B8
:10220000A2089ECF83E38C0F833108F099CF61E061
:102210008C2F46D895CF8C2F0E94E30827DCC8CF9F
:10222000CF93DF93EC01805E9109089720F06AE973
:1022300071E1209711F46EE871E1CE010E94ED0387
:102240008C2F65DFDF91CF910895811509F44FC080
:10225000823861F40E94670881FF49C089E30E94C7
:10226000CA0804DC89E30E94E30800CC833851F4F7
:102270000E94670880FF3BC083E50E94CA08F6DB26
:1022800083E5F1CF843851F40E94670882FF2FC0A4
:1022900087E40E94CA08EADB87E4E5CF9CEF980F49
:1022A000913A08F390E2980F983050F4877091E0DB
:1022B00001C0990F8A95EAF7892F0E94DB04D5CFD8
:1022C0009BE5980F933020F480E090E00C947A081E
:1022D00098E5980F9B3120F480E090E00C94A208E0
:1022E00093E3980F933118F460E00C94500908952B
:1022F0001F93CF93DF93182FEB0109DF209731F461
:10230000812FA3DFDF91CF911F9108958FE99FE087
:102310000197F1F700C000002197F0CF811519F067
:102320000E94D504A3CB0895811519F00E94DB0407
:102330009DCB0895811531F09091A903892B80934D
:10234000A90394CB0895811539F080959091A90344
:1023500089238093A9038ACB0895809194028115E3
:1023600021F082E2F0DF109294020895CF93DF9380
:10237000EC014A855B856E857F850E9462089B81A2
:1023800090958091A90389238093A9038C810E9451
:10239000DB046CDB86E0FE0111928A95E9F7DF91A0
:1023A000CF910895CF93DF93EC018D8181FD13C010
:1023B00082608D838091A9039B81892B8093A903DF
:1023C0008C810E94D50452DB488559856E857F85B6
:1023D000CE010E94620810929E0310929D038D818F
:1023E00080FD02C0CE01C2DFDF91CF9108951F931F
:1023F000CF93DF93182FA0911303B091140310977C
:1024000009F449C010921603109215031092990214
:10241000109298021696CD91DC911797CE019A955D
:1024200081159F4108F4D07ED1E0C11101C0D0E0F8
:102430001996ED91FC911A97309731F01B966D919A
:102440007C9180E00995D823D11539F08CEF8C0F61
:10245000813A28F58C2F0E94E3081115A9F0E0912C
:102460001303F0911403808584FD0EC08091120344
:10247000811551F0808191819C01215031092F33C8
:102480003E4710F40E942F0AF1DA109214031092C2
:10249000130310921203DF91CF911F910895E6DA92
:1024A0008C2FD3DEDACFAFE0B0E0E9E5F2E10C94B7
:1024B000C930FE0131968AE0DF011D928A95E9F765
:1024C0008AE4E82E81E0F82E8F019FE4C92E91E086
:1024D000D92E3F01AA24A394B12C35E5832E31E0F7
:1024E000932EF70181917F018F3F09F43EC0F8944C
:1024F000E82FE295EF70F0E021A18F70A50102C0F6
:10250000440F551F8A95E2F7CA01922F982B91A389
:1025100092A18095892382A3789400C0EFE4F1E032
:1025200031E0512C21912F3F79F0A22FA295AF706D
:10253000A05EB0E08C9190E02F7002C095958795D9
:102540002A95E2F780FF7BC080E0582A330F8E1671
:102550009F0641F7F70182918F3F11F00E94DF063D
:1025600050EA5A95F1F7D8015C920F5F1F4FCE14D5
:10257000DF0409F0B6CF4AE050E0B3018FEF91E0FD
:102580000E9484319C01892B41F08AE0F301AFEF76
:10259000B1E001900D928A95E1F700910A0210E0F6
:1025A000075D1D4F232B09F44CC081E08093D701B8
:1025B0000E94F2089093D6018093D5018091520237
:1025C000811509F498C07E01BBE0EB0EF11C85E09B
:1025D000F70111928A95E9F78091D8018A3008F0C5
:1025E00054C04CEB54E1B701C80199D9811509F4E5
:1025F00070C041E654E1B701C80191D9811509F4D1
:1026000068C049E555E1B701C80189D9811509F4C8
:1026100060C01092D8018091090290E045E050E03E
:10262000B701875D9D4F0E94843121E02093D40142
:10263000892B09F041C02F96EFE00C94E530832FF1
:1026400084CF8091D701811509F4B8CFE090D501EE
:10265000F090D6010E94F2088E199F09059708F4A0
:10266000ADCF45E050E06FEF71E0C8010E948431CA
:10267000892B41F085E0EFEFF1E0D80101900D9258
:102680008A95E1F71092D70199CFC090D201D090EE
:10269000D3010E94F2088C199D09843F914008F0F3
:1026A000A0CF8091D401811531F285E0D7011D9230
:1026B0008A95E9F71092D401A0910902B0E0A75DD4
:1026C000BD4F85E0FE013B9601900D928A95E1F7A2
:1026D000B2CF8091D8018F3F39F40E94F2089093D5
:1026E000D3018093D201DDCF8F5F8093D8018A30F0
:1026F00008F491CFF2CF85E0F801AFE3B2E00190AA
:102700000D928A95E1F78FE392E00E94470B809348
:102710003E02C0904402D0904502E0904602F09004
:1027200047028091CE019091CF01A091D001B0914C
:10273000D101C816D906EA06FB06B1F0C092CE0157
:10274000D092CF01E092D001F092D1010E940B0A09
:10275000C61AD70AE80AF90AC0925402D092550262
:10276000E0925602F0925702809148020E948A0736
:1027700062CFA0E0B0E0EFEBF3E10C94CF30EC01DE
:102780008881811509F1813009F045C08981813046
:1027900051F48A81239660E570E0893311F060E09E
:1027A00070E0A6DDEDCF823021F48A812396AFDC84
:1027B000E7CF833021F48A81239647DDE1CF84304F
:1027C00041F022968111DCCFCDB7DEB7E9E00C9461
:1027D000EB308A81239620E030E09AE0682F605346
:1027E000770BAB016A30710560F02115310551F3AB
:1027F000EFE9FFE03197F1F700C000002150310907
:10280000F4CF929FB001939F700D11249A01260F6F
:10281000371F8991E3CFE82FF0E0E354FE4FB490E7
:10282000282F26952695269530E0F901E355FE4F91
:10283000E4908770F12C082E02C0F594E7940A9476
:10284000E2F7E0FAEE24FF24E0F8F901E356FE4F48
:10285000C490D12C082E02C0D594C7940A94E2F7F4
:10286000C0FACC24DD24C0F8F901E357FE4F0491EF
:1028700010E002C0159507958A95E2F701701127BF
:10288000E114F10411F081EE42DCC114D10411F025
:1028900086EE3DDC60E070E08B2D2ADDC114D104B2
:1028A00011F086EED2DCE114F10411F081EECDDC02
:1028B0000115110521F060E070E08CE219DD219630
:1028C0005FCFCF92DF92EF92FF921F93CF93DF9370
:1028D00000D000D0CDB7DEB7C0903A02D0903B0216
:1028E000E0903C02F0903D020E940B0A6C197D09B9
:1028F0008E099F0911E0643671058105910578F113
:102900000E94170ADC01CB010296A11DB11D89832B
:102910009A83AB83BC838091220190912301825CD6
:102920009D4F20912101422F50E0253010F044E0CE
:1029300050E0BE016F5F7F4F0E94913182E090E0D6
:102940000E945830182F811551F00E940B0A609395
:102950003A0270933B0280933C0290933D02812F98
:102960000F900F900F900F90DF91CF911F91FF90DC
:10297000EF90DF90CF9008958F929F92AF92BF9289
:10298000FF920F931F93CF93DF9300D000D000D01E
:10299000CDB7DEB7F62E072F80E090E00E945830CA
:1029A000182F811509F460C080911401482F50E060
:1029B000811511F041E050E0609115017091160110
:1029C000625C7D4FCE0106960E94913180904E024E
:1029D00090904F02A0905002B09051020E940B0ABA
:1029E000681979098A099B09643671058105910581
:1029F00038F48FE392E00E94470B9E818917A1F182
:102A000081E090E00E9458308115C9F180911C014D
:102A1000482F50E0863010F045E050E060911D01F5
:102A200070911E01625C7D4FCE0101960E94913132
:102A30008FE392E00E94470B9E81891320C00E9481
:102A40000B0A60934E0270934F0280935002909352
:102A5000510285E0FE013196A9E4B2E001900D92A9
:102A60008A95E1F781E00CC085E0EFE3F2E0DE015A
:102A7000119601900D928A95E1F71111EACF80E04D
:102A800095E0E9E4F2E0AF2DB02F01900D929A9518
:102A9000E1F70F900F900F900F900F900F90DF9134
:102AA000CF911F910F91FF90BF90AF909F908F900B
:102AB0000895A1E0B0E0EFE5F5E10C94D03010917D
:102AC000930210FF43C01695169516951983009131
:102AD0004802C0903602D0903702E0903802F09061
:102AE00039020E940B0A6C197D098E099F09643610
:102AF00071058105910510F4011719F180912A01E2
:102B000090912B01825C9D4F20912901422F50E032
:102B1000211511F041E050E0BE016F5F7F4F0E9430
:102B2000913183E090E00E945830811559F00E9465
:102B30000B0A6093360270933702809338029093A9
:102B4000390281E02196E8E00C94EC3010E0BECF31
:102B500086E090E00E94B1318093930282FD07C02D
:102B60008DE38093930283E992E00E94DC0C8091D4
:102B70009302803420F08770886380939302909151
:102B80009302892F817090FF04C0892F86958695C6
:102B900086950C94F8060F931F93CF93DF9386309E
:102BA00030F56A3020F5463010F5C42FD0E0CC0F58
:102BB000DD1F2CE0629FC00DD11D112438E7839FDB
:102BC000C00DD11D1124CE0189960E94B131082F6C
:102BD00010E0102F0027CE018A960E94B131980193
:102BE000282BC901DF91CF911F910F91089580E0AB
:102BF00090E0F8CF462F672F20915A0230915B0268
:102C0000232B81F4703F39F4403F61F480915802E6
:102C10009091590208957A3028F4463018F486309D
:102C200008F4B9CF80E090E00895A0E0B0E0EBE1D7
:102C3000F6E10C94D1307C010091A8038091A703A8
:102C4000082BC5E0D0E010E0C8010C2E02C095951D
:102C500087950A94E2F780FD09C02197A8F7D12C47
:102C60008D2DCDB7DEB7E7E00C94ED30DC2EB7014B
:102C70008C2FC0DF0E94E105019779F3F1CF0F930C
:102C80001F93CF93FC01858100811181811581F013
:102C9000611571F0C801C9DFC82F682FC8010E94F3
:102CA0002704B8018C2FA6DFCF911F910F910895B3
:102CB000C8010E945D04C82FF4CFCF93DF93D82FB3
:102CC000C92FB3DF6D2F7C2F95DF0E94E105DF91C7
:102CD000CF910895FC018481811599F080819181C3
:102CE000ECDF282F92959F70963099F060F4925FF8
:102CF0009F70923030F4203FB1F038F481E0283EEC
:102D000038F080E008959A5FF3CF81E0243FC9F75F
:102D1000089591E0213F09F090E081E0283E08F01D
:102D200080E0892B089581E00895382F292FCB0169
:102D3000A32FB22F87369105A105B10520F4875640
:102D40009C4F0C94B13180E0089585E290E00E94A0
:102D5000B131863389F486E290E00E94B13185304A
:102D600059F487E290E00E94B13191E0873209F096
:102D700090E0892F8170089580E0FCCFAAE0B0E058
:102D8000E4ECF6E10C94CB30C0903302D0903402E6
:102D900081E090E09093340280933302812C912C57
:102DA000E12C5401F12C15C0F80125913591472DE6
:102DB0006F2D8E2D0E94F80C0E5F1F4F739486E0CE
:102DC0007812F2CF96E0A90EB11CF394EAE0FE1659
:102DD00039F08501000F111F04501D4F712CE4CFF5
:102DE000E394FCE38F0E911C86E0E812DACF1A829E
:102DF00019821C821B821E821D8218861F8288EC0B
:102E000090E09A87898709EF12E0FE0131967F01F1
:102E10004AE050E0B801C7010E94EB31065F1F4F46
:102E200057010934F3E01F0799F789E0F701119280
:102E30008A95E9F78FEF9FEF9E838D8387E08A87DE
:102E40004AE050E0B801C5010E94EB31065F1F4F18
:102E50000939F3E01F07A1F7D0923402C092330280
:102E60002A96EDE00C94E730AAE0B0E0EAE3F7E15F
:102E70000C94CE300AE912E089E4E82E83E0F82EC3
:102E800097E0B92E26EFC22E21E0D22EAA24A394D9
:102E90004AE050E0B701CE0101960E94A131F8014D
:102EA0003896DF018B2D1D928A95E9F789819A81E9
:102EB000D80111969C938E938F8112968C931297C2
:102EC0008D8113968C931397888514968C93149701
:102ED000898515968C9315978B819C8117969C9369
:102EE0008E9316978A8587FD04C01E96DC92CE923B
:102EF0001D9780FF02C0F801A08681FF07C0D8019E
:102F000018969C911897926018969C9382FF04C023
:102F1000F80190859460908783FF07C0D8011896C8
:102F20009C911897986018969C9384FF04C0F801B0
:102F300090859061908785FF07C0D80118968C9185
:102F40001897806218968C93BAE0EB0EF11C015F23
:102F50001F4FE9E9EE16E3E0FE0609F099CF2A9645
:102F6000EAE00C94EA30282FCB01283070F44AE0D4
:102F7000249F90011124B90167507D4F4AE050E031
:102F80000E94A13180E090E008958FEF9FEF0895B7
:102F9000AAE0B0E0EEECF7E10C94D6309C01975536
:102FA0008115914068F4BE016F5F7F4F822FDBDF98
:102FB000892B31F489859A852A96E2E00C94F230C7
:102FC00088EC90E0F9CFA0E0B0E0E9EEF7E10C94F6
:102FD000D130162FD72FC42FD22E8115A1F04093B8
:102FE000A1030E94F2089093DA018093D901C7707F
:102FF00081E001C0880FCA95EAF790D9CDB7DEB756
:10300000E7E00C94ED309091A103491335C0E090B6
:10301000D901F090DA010E94F2089C012E193F09B3
:103020007901812F9D2FB4DFE816F90628F5D0E24B
:10303000DD0DCD1591F0C77011E0812F01C0880F13
:10304000CA95EAF771D9D83040F48D2D877001C048
:10305000110F8A95EAF7812F61D960E070E0802F27
:1030600047D9D83058F62D2D277081E001C0880F40
:103070002A95EAF759D9C2CFC77081E001C0880FFD
:10308000CA95EAF7F7CFACE0B0E0E9E4F8E10C94D8
:10309000C7307C01DC0114968C91811509F4F4C0D1
:1030A00061E0C701ECDD8C01F7018581811521F11B
:1030B00080919D0390919E030097F1F008171907E6
:1030C000D9F0FC01FF27887F9927892B09F089C057
:1030D000A4E0EE0FFF1FAA95E1F7E35EFC4F8581A8
:1030E0008460858311830083CF015CD91092A9038A
:1030F00061E0C701C4DD8C010034F2E51F0709F46B
:1031000083C008F071C0043232E5130709F49CC093
:10311000053242E5140709F4A0C0033252E5150751
:1031200009F481C0D70115968C91811509F488C1E5
:10313000C80197578038910508F033C1003208F074
:1031400093C066E670E080E090E0EFDD81118CC016
:10315000812C912C540101119FC004E09E012F5F2E
:103160003F4F6901D601E02F1D92EA95E9F724014E
:103170003501FFEF4F1A5F0A6F0A7F0AC501B401DC
:10318000D4DD8983811509F46FC0813009F006C14F
:10319000A50194012E5F3F4F4F4F5F4F2D833E831C
:1031A0004F835887C301B201C0DD182F8A83811570
:1031B00009F45AC08FEF810F833008F084C06D810D
:1031C0007E818F819885B1DD8B83811511F0C601D9
:1031D000D0DA2401350133E0430E511C611C711C0F
:1031E000A0C0E0E0F0E07BCF013482E51807A9F051
:1031F000023492E5190709F095CFD70115968C9105
:10320000811591F182E006C0D70115968C91811548
:1032100059F180E00E94C90C27C0F7018581811512
:1032200019F181E0F7CFF7018581811549F083E03D
:103230000E940F0445E064E083E00E94910414C002
:1032400083E00E941904F6CFD70115968C91811561
:1032500011F084E0EDCF84E0F4CFF7018581811592
:10326000B9F085E00E940F048091AA038770811550
:1032700059F0F7018581811539F08091F10382FFC2
:1032800003C082E00E94BA042C96E1E10C94E33082
:1032900085E00E941904E8CFB7E68B169104A104DB
:1032A000B10411F3C501B40140DDEFEF8E1A9E0A9F
:1032B000AE0ABE0A8111F0CF01504DCF4D805E8025
:1032C0006F8078842EC08BEF810F833098F52401B6
:1032D000350143E0440E511C611C711C6D817E81DF
:1032E0008F81988522DD8B838115D9F0C301B201CE
:1032F0001CDD8C83811571F08B819C8181305FEFA7
:10330000950710F0982F8827163071F0173079F054
:103310000E944C252401350134E0430E511C611CF0
:10332000711C530142011ECF0E94F924F3CF0E9469
:103330001A25F0CF143009F0C1CF6D817E818F81C5
:103340009885F3DC182F2401350184E0480E511CC8
:10335000611C711CC501B4016D5F7F4F8F4F9F4F82
:10336000E4DC111509F480CF811509F47DCF81507B
:10337000990B4FEF489F9001499F300D1124A12FC9
:10338000A150BB0B2A0F3B1F2150310950F2EFE92E
:10339000FFE03197F1F700C00000F6CFC601E9D990
:1033A000C0CF033028E7120709F4B0C070F5013030
:1033B00048E7140709F4A8C0023058E7150709F4D4
:1033C000D4C0011588E7180709F496C0023AF2E55F
:1033D0001F0709F06CC021EE30E02770332781E031
:1033E00090E001C0880F2A95EAF72091970230916A
:1033F0009402311509F408C1F7013581311509F43A
:10340000FEC0282B209397022FCF043098E719078E
:1034100009F48CC00530A8E71A0709F4B8C00337CF
:10342000BCE71B0799F6F7018581811509F41CCFCC
:1034300080919402811509F4BCC00E94AD1114CF93
:103440006801B7E5DB1AC114E1E0DE0640F769E880
:1034500072E08C2D88DD892B21F5C601E4E0880F10
:10346000991FEA95E1F7FC01E35EFC4F22812130D0
:1034700081F52091890230918A02232B91F02091CD
:103480008B0230918C02232B61F020918D023091C0
:103490008E0240918F0250919002242B352B232BCA
:1034A00001F1D70115968C91811509F48FCF033A5C
:1034B00022E5120708F08DC0C80190528115904294
:1034C00008F48EC0013E110509F485CF053E1105B3
:1034D00083C0223031F720918D0230918E02232B50
:1034E00001F3FC01EE5DFC4F20812E7F2083835E83
:1034F0009C4F0E94D211D5CF87E00E948A0783E9B2
:1035000092E00E94DC0CB0CE80E0F7CF8091930275
:10351000883028F188508093930291E0883008F435
:1035200090E08091930290FB80F913C090919302F8
:10353000892F869586958695983340F48F5F880FFE
:10354000880F880F9770892B809393028091930244
:1035500081608093930283E992E00E94DC0C809169
:1035600093028695869586950CC08091930280FF84
:103570000BC08E7F8093930283E992E00E94DC0C63
:1035800080E00E94F80670CE0E94E20C6DCE809121
:1035900093028695869586958F5F8F71883008F0A7
:1035A00080E0880F880F880F909193029770892B85
:1035B000B2CF1092A5030E94E3040E94F20888573C
:1035C0009C4E909396028093950281E080939402A2
:1035D0004BCE023B42E5140741F525EE30E0FDCE2F
:1035E000D70116968C91803100F5812F99278F7124
:1035F00099278230910509F4EECE4297EDCF809560
:1036000082238093970230CE322F3823311569F010
:10361000982F90959223909397020E94DB04D701F4
:1036200015968C91811509F41FCE80919402811515
:1036300009F467C0C090A503D090A4030E94F208CB
:1036400088579C4E9093960280939502F70185814E
:10365000811509F456C08D2D8C298D79811184C076
:103660000115F0E51F0700F5011520E4120708F029
:1036700082C0063E110509F444C0C801905281156C
:10368000904208F07FC0D70116968C91803108F4E3
:1036900063C0C80199271092A9038D329105E9F4FE
:1036A00082E08093A90372C0003EB2E51B0708F0D8
:1036B00046C0003CE2E51E0720F5003AF2E51F0790
:1036C000E0F4003622E51207E0F4C8019255803498
:1036D0009105B8F01092A903C8018E32910508F047
:1036E00062C08832910508F04FC08E31910508F014
:1036F0004DC004974A97A0F237C0043B32E5130748
:1037000049F7F7013580311409F457C00E35FCE74D
:103710001F0709F44EC00F352CE7120751F00D3585
:103720003CE7130709F049C080913101811509F484
:1037300040C01092310180E00E94F71195CD093709
:103740004CE7140728F407375CE71507D0F6C2CF1B
:103750000B378CE71807D4CF812F8F71843189F212
:10376000863111F41092A9030E94AD118091970245
:103770000E94D504C6CFD70116968C91803108F0EF
:1037800088CFBFCFC80187CF8A9771F78091970202
:10379000811531F08091A90392E089278093A903D4
:1037A0000E94360DAECF8C34910581F38D3292405C
:1037B000ECCF81E08093310157CD809131018111AF
:1037C00069C0C80197558115914008F0FFC05801A4
:1037D000F8EFAF22BB24A114B10409F045CDF801E4
:1037E000FF2754E0EE0FFF1F5A95E1F79F01235E7C
:1037F0003C4F6901D70115968C91EE5DFC4F90818D
:1038000080FB90F99083811509F4D9C10E94F208D8
:103810009093A00380939F03F60182818F5F828340
:103820008091A9039091A503892B83838091A403A0
:1038300084834681578166857785C6010E94620828
:10384000D60115968C9181FF5801B0929E03A092EB
:103850009D03D70115969C91911509F401C610920C
:10386000A103980130572332310508F007C684E0E0
:1038700090E00E94B9319093F1038093F003F80136
:10388000E150F047E232F10508F0E1C1EF5DFD4C97
:103890000C945531380150EE651A71085090A6030A
:1038A0008091A503582A8091A403582A88E06816BD
:1038B000710408F05EC098012770332781E090E022
:1038C00001C0880F2A95EAF7311409F44FC0582A2D
:1038D000D7018D919C910E945D0421E030E0F901B7
:1038E00002C0EE0FFF1F8A95E2F7FC87EB8720915D
:1038F0001303309114033E832D8340911B03509199
:103900001C035A8749876AE9C62E62E0D62EA12C8D
:10391000B12C511005C0D60112968C9181111BC09B
:10392000F601838190E02B853C8582239323892BAC
:1039300091F08085982F9770911101C087E038E051
:103940006316710408F066C0311409F45FC08695EF
:103950008170811164C09FEFA91AB90AAFE0CA0E45
:10396000D11CB8E0AB16B104A1F61CC0809558225A
:10397000AFCF311038C080911B0390911C03081702
:10398000190781F410921C0310921B031092170365
:10399000109218031092190310921A031092160332
:1039A000109215038091130390911403009709F46A
:1039B00008CFE8E06E16710408F0EBC0652D0E9498
:1039C000C707811103C081E00E94F711F7018581CB
:1039D000F801E851FC47E730F10508F03ACFED5B1C
:1039E000FD4C0C94553110931C0300931B030E9453
:1039F0000B0A609317037093180380931903909335
:103A00001A03109216031092150362CF82FB8827C7
:103A100080F99FCF311409F49ECF80FF9CCFD6014F
:103A20008D909C900815190519F4311409F493CF61
:103A3000ED81FE81EC15FD0509F48DCFD6011D96B3
:103A4000ED91FC91309721F08081811509F483CFAD
:103A5000652DC6010E94C707811509F47CCF81E05E
:103A60000815190509F080E0482E432081149104BF
:103A700041F0411006C0E985FA858E169F0609F0CF
:103A80006ACF80E00E94F711D0921403C092130312
:103A900081E0809312038FE08A9DF0018B9DF00DF1
:103AA0001124E656FD4F85818093990241100EC086
:103AB0008114910459F0808191819C012450310935
:103AC000213A310508F049C00E94E3088FE08A9D41
:103AD000F0018B9DF00D1124E656FD4FC680D78076
:103AE000C6019A9581159F4110F420EED2229924A7
:103AF0009394C60101978F339E4708F0912C8FE075
:103B00008A9DD0018B9DB00D1124A656BD4F1996EC
:103B1000ED91FC911A97309731F01B966D917C9145
:103B200081E0099598229114A9F08FE08A9DF00117
:103B30008B9DF00D1124E656FD4F868197810E94E2
:103B4000C30380939802C60148E06416710440F4F0
:103B50000E942F0A0E94360D0AC00E942511B6CF7E
:103B60000497813A910548F48C2D0E94CA084114AB
:103B700009F427CE0E94360D77CB0E94360D8FE3D5
:103B80009CE90197F1F700C000008C2D0E9487107E
:103B9000EECFDC012D913C910217130741F4311057
:103BA00009C01092120380E00E94F7110ACE31146E
:103BB00009F407CEFC01808585FD03CEF4CFF90121
:103BC0004485558566857785C9010E946208D601BE
:103BD00015968C9181FF3DCEC6010E94B611809151
:103BE0009D0390919E030817190709F032CE109299
:103BF0009E0310929D032DCE06E221EE41EE6AE176
:103C00007CE7E1D931CB07E225EE45EE6BE17CE7BD
:103C1000F8CF06E221EE40EE68E17CE7F2CF07E262
:103C200025EE44EE69E17CE7ECCF06E221EE42EEC0
:103C30006CE17CE7E6CF07E225EE46EE6DE17CE73E
:103C4000E0CF08E221E045EE6EE17CE7DACF80913B
:103C5000F00381608093F0036091F0037091F103B1
:103C600084E090E00E94E7310E948C0DFDCA8091B3
:103C7000F10388608093F103EFCF8091F0038260BD
:103C8000E9CF8091F0038460E5CF8091F0038860F4
:103C9000E1CF8091F1038160EDCF8091F1038260EB
:103CA000E9CF8091F0038061D5CF8091F0038062ED
:103CB000D1CF8091F0038064CDCF0E948C0D809194
:103CC000F0038068C7CF8091F0038C60C3CF8091F0
:103CD000F1038360CFCF8091F0038E7FBBCF8091C3
:103CE000F103877FC7CF8091F0038D7FB3CF8091A1
:103CF000F0038B7FAFCF8091F003877FABCF8091B4
:103D0000F1038E7FB7CF8091F1038D7FB3CF809188
:103D1000F0038F7E9FCF8091F0038F7D9BCF8091AA
:103D2000F0038F7B97CF0E948C0D8091F0038F77EB
:103D300091CF8091F003837F8DCF8091F1038C7FB1
:103D400099CF8091F003992782FF939590FB82F998
:103D500090FB83F97FCF8091F103982F909590FB92
:103D600080F990FB81F986CF9091F003892F8F7BAA
:103D700096FF80646FCF0E948C0D9091F003892F85
:103D800097FB87F9805866CF61E08EE090E00E9453
:103D9000CD3162CF60E0F9CF9091F003892F8F7E13
:103DA00094FF806157CF9091F003892F8E7F90FF11
:103DB000816050CF9091F103892F877F93FF8860B6
:103DC00059CF89E26DC389E256C30737BCE71B07A9
:103DD00079F00837ECE71E07A1F09801205E324524
:103DE0002032310598F4911111C0802F8F7112CAC1
:103DF00081E0911541F00E940F0443E062E081E010
:103E00001CCA82E0F6CF0E941904F7CF4091A303A9
:103E10008091A803282F30E02095309570E024236E
:103E20003723232B19F048234093A3030B37FCE7D8
:103E30001F0741F4911509F417CA0E94F6030E9466
:103E4000E80712CA003422E5120708F055C0003214
:103E500032E5130708F057C0011540E5140750F587
:103E6000011550E4150708F064C0911509F47AC0F3
:103E70000A35BCE71B0709F4DDC008F0C2C00130F9
:103E8000FCE71F0709F4D4C003302CE7120709F43C
:103E9000C9C001151C4709F065C00E948C0D8FEF49
:103EA00094E3ACE081509040A040E1F700C00000F6
:103EB0000E94090C9801305521153240B0F6980146
:103EC00045E0369527954A95E1F7822F8F7020912E
:103ED000A30330E041E050E0082E02C0440F551F1C
:103EE0000A94E2F724233523232B09F4BECF911142
:103EF000A6CF1092A5033ECE9801205C3245203219
:103F0000310508F0B2CF802F8F712091A30330E0EC
:103F100041E050E0082E02C0440F551F0A94E2F71A
:103F200024233523232B09F4A0CF911509F49CC930
:103F300086CFD70116968C91803108F096CF9111DB
:103F400011C0212F2F7081E090E002C0880F991FCF
:103F50002A95E2F72091A30330E082239323892B53
:103F600009F082C9D70115968C911597CD90DC90F8
:103F7000811509F463C0C6010E941516182F682F19
:103F8000C6010E942704B601812F0E94FA150E94E3
:103F9000E1058C01F701B580A680A2942FE0A22252
:103FA0008091AA038770811501F1CB2CB114F1F037
:103FB000812F807F803461F080E2800F8830A8F00C
:103FC000812F807E803221F4023078F0A11469F0D4
:103FD0008091F10382FF09C082E00E94BA048091BF
:103FE000AA038770CC24C3948111C12CE12FE295E0
:103FF000EF70103C08F082C0F0E0E65BFD4C0C94E2
:1040000055310B354CE71407B9F08091F1030024CA
:1040100082FF0394802D0C351C4709F0A3CF0E942A
:104020001F0DA0CF6FEF7FEF80E090E00E94E7319F
:104030000E94AF0D81E0F3CF80E0F1CFC6010E9476
:104040005D04182FA0CFF12FFF70DF2E103118F074
:10405000D29490EFD922B114A9F0D11459F080E292
:10406000800F883010F0011107C08D2D0E94D504FB
:104070000E94360D802F40C08091A9038D29809326
:10408000A903F6CF802F0E942511D114B9F180E247
:10409000800F883010F0011104C08D2D0E94DB04C8
:1040A00006C0D0948091A9038D218093A9030E941A
:1040B000360D24C0212F2F70D22E107F103219F010
:1040C000D29480EFD822011549F0013009F483C061
:1040D000B11409F48FC0A114A9F1CCCF8091F103E0
:1040E00082FD2CC0B11421F1D11429F08D2D0E9434
:1040F000D5040E94360D80E00E948710C11409F497
:10410000D9C08091AA0380FDD5C0D70115961C9215
:104110008695869586950E940F04C7010E944318D4
:104120008091AA038695869586950E941904C2C03F
:1041300080E00E942511D11409F3AFCFB11469F1C9
:10414000A11004C08D2D0E948E11D8CF31E0A31292
:1041500010C01091A4038D2D8123D81679F20E94EE
:10416000F2089093AE038093AD031D291093A4032E
:10417000C5CF45E0A412C2CF8D2D0E948E118D2D8A
:104180000E9412098091A6039D2D9823D91609F447
:10419000B5CF8D298093A603B1CFA11012C08D2D6C
:1041A0000E9494118D2D0E9412098091A6039D2DCD
:1041B0009823911509F4A2CFD094D822D092A603C7
:1041C0009DCF51E0A5129ACF8091A5038D21811535
:1041D00009F494CFE4CFB11429F086E0A81608F0D2
:1041E0008DCFB0CF95E0A91608F088CF8D2D0E9415
:1041F000941184CFA114D1F3093349F4AFEFB7EE92
:10420000E3E0A150B040E040E1F700C00000802FA3
:104210000E94251173CF812F869586958370811515
:1042200061F0813009F06ACFC8019370B11002C00B
:1042300080E090E00E94A20861CFC8019370B110A5
:1042400002C080E090E00E947A0858CF6B2D802F4A
:104250000E94500953CF812F8370811139C0B11052
:1042600027C0402F429546954770440F440F802F3A
:104270008F70042E01C0880F0A94EAF7202F207156
:1042800004FF07C02FE030E001C0220F4A95EAF793
:1042900020951695169513701230A9F0133089F0F9
:1042A0003091A703113061F0822B83230E9409040F
:1042B0000E94670860E0C7010E943F160C944419F1
:1042C000832B822BF3CF822B9091A7038927EECFEC
:1042D000B11451F110FFECCF402F42954695477035
:1042E000440F440F802F8F70042E01C0880F0A9452
:1042F000EAF7202F207104FF07C02FE030E001C053
:10430000220F4A95EAF720951695169513701230EC
:1043100089F0133069F03091A803113041F0822BFD
:1043200083230E940C04C4CF823010F2D5CF832B9C
:10433000822BF7CF822B9091A8038927F2CF1F7091
:10434000B11439F0812F0E940F04802F0E948E112A
:10435000AFCF802F0E949411812F0E941904A8CF03
:10436000023F71F170F4003FC9F0013F91F0B114C8
:1043700009F465C0A11409F45FC0802F0E94871062
:1043800097CF033F21F1043F91F78091F10382FD24
:104390002AC0812F8F71B11401F316C0B11469F0D6
:1043A000F5E0AF1608F084CF1F7181E090E0012E98
:1043B00001C0880F0A94EAF7BECF26E0A216F2CF1A
:1043C000812F8F71B110C9CF0E940F0471CF80E08F
:1043D000B11409F4A6CF1F7181E0012E01C0880F2E
:1043E0000A94EAF79ECFB114C1F08091AA038770B6
:1043F000843049F41092AA031092AC031092AB03DC
:10440000812F8F71AACF35E063E0A31608F050CF5B
:10441000812F8F710E94FE084BCF45E0A41640F01B
:104420001092AA031092AC031092AB0364E0F0CF99
:1044300081E00E94BA043CCF812F8F71C5CFA114B7
:10444000F9F2093349F45FEF87EE93E05150804071
:104450009040E1F700C00000802F0E94251128CF76
:104460000631BCE71B0709F0B0CC8091A20381158F
:1044700009F4A9CC85E30E94E3087CCB0631ECE784
:104480001E0709F0A2CC8091A5038A7A91E08111E0
:1044900001C090E09093A203811509F492CC85E3CA
:1044A0000E94CA0867CBA0E0B0E0E9E5F2E20C9414
:1044B000D1308091EF03803108F049C08091EE0344
:1044C000811509F444C0C091B00387E0D82E8091D3
:1044D000AF038C17E1F1EC2EF12CDC9EE0011124EE
:1044E000FE01EF54FC4F84818115B1F191818091DF
:1044F000EA03981331C090818091E90398132CC08E
:104500008581811129C0028113818091EB039091F3
:10451000EC03081B190B60E089EE93E00E943F1644
:104520000E94C81708171907B8F48091EF038F701D
:1045300080618093EF03C954DC4F88818F70806164
:10454000888389EE93E00E9443180E94B004CDB79F
:10455000DEB7E7E00C94ED30E7012196C770B7CFE6
:10456000ADE0B0E0E6EBF2E20C94C9308C0186E0FD
:10457000F801DE01189601900D928A95E1F7F80195
:10458000F580E48089EE882E83E0982E8091ED03FB
:10459000811117C0E11491F0F11409F455C1C8015B
:1045A0000E946A16811509F44FC187E0F801A9EE4F
:1045B000B3E001900D928A95E1F775DFFF24F39443
:1045C00061C0A280B380D090EE038091EB03909104
:1045D000EC033501681A790AD11409F4F0C0C080DF
:1045E000518060E089EE93E00E943F160E94C81758
:1045F0006816790608F09EC0E11401F38091EA0381
:10460000F8019181E090EF03F0E1EF1608F05BC054
:10461000981317C09091E903F8018081981311C095
:10462000F1104BC08E2D8F7080618093EF0389EE67
:1046300093E00E9443188091EF03F8018683F12CE8
:1046400021C0F1103AC040E0652D8C2D0E94EA0B8C
:1046500040E0652D8C2D0E94EA0BF82E8111EFCFE2
:10466000888599850E945D16292F22952F70903498
:1046700070F49F702230A0F09115B1F0F80196818E
:10468000903190F48F2D2D96EFE00C94E5302A5F59
:104690002F70223068F0C8010E944318FD2CF2CF21
:1046A000911511F0811571F3805E883058F3F3CFC6
:1046B000803F40F3815F8330F9CF8091EF038160C9
:1046C0008093EF03BCCF981315C09091E903F801D4
:1046D000808198130FC0F1100DC0E682C8010E94BE
:1046E000431887E0F801A9EEB3E001900D928A9596
:1046F000E1F764CFC8010E946A16811509F4A4C0CD
:10470000F11409F4A1C08091EF03803208F44DCF79
:104710008091E9039091EA039A838983BC82AB82FA
:104720008091ED038D831E82EF82CE0101960E945F
:1047300043183BCFD090EF03F0E1DF1650F489EE41
:1047400093E00E94431887E0F40111928A95E9F7FB
:1047500076CFE11409F432CF9091EA03F801818118
:10476000981311C09091E903808198130CC0F11047
:104770000AC0D682C8010E94431887E0F401119252
:104780008A95E9F71BCFC8010E946A16811509F4C2
:104790005BC0F11409F458C08091EF03803208F433
:1047A00004CF8091E9039091EA039A838983BC82C4
:1047B000AB828091ED038D831E82DF82B6CF60E0F5
:1047C00089EE93E00E943F160E94C817681679068A
:1047D00008F0B9CFE11409F4F1CEF114A9F19091E8
:1047E000EA03F8018181981325C09091E903808143
:1047F000981320C08091EB039091EC03A81AB90A9A
:10480000F8ECAF16B10408F06CCF8091EF0380FD97
:1048100068CF803108F465CFF8018683982F907FA8
:10482000903F09F45BCF982F907F905F8F70892B1A
:10483000868354CFC8010E946A168111B6CE80913A
:10484000EF0381608093EF03C8010E944318B6CE46
:10485000ABE1B0E0EEE2F4E20C94D4304E8B5F8B2F
:10486000688F798F8A8F192F9B8F91111092A903CE
:104870001D8A86E0FE017696DE011F9601900D925C
:104880008A95E1F70A8D8091F10382FF1FC00E9493
:10489000F2082091AB033091AC03821B930B883854
:1048A000934138F08091AA0382FD03C082E00E9408
:1048B000BA040E94F2082091AD033091AE03821B2E
:1048C000930B8838934110F00E94E304011561F0C6
:1048D0000B8B1C8B61E0CE010F960E943F1661E0AE
:1048E000CE010F960E943F160B8B1C8B87E0FE01BA
:1048F0003F96DE01189601900D928A95E1F7CE0160
:1049000008962EDE811110C02091AF033091B003C4
:1049100087E0FE013896DE01119601900D928A958E
:10492000E1F78C8581110BC017E08091B003909165
:10493000AF0389132BC06B96E4E00C94F030822F08
:1049400090E00196877099273817190671F40E9434
:104950008C0D1092AF031092B00387E0E9EEF3E004
:10496000DF011D928A95E9F7DFCF97E0929FD00192
:104970001124AF54BC4FFE01319601900D929A95CF
:10498000E1F78093AF030E94B004CECF189FC0011F
:1049900011248F549C4FE4DD811569F28091B0039E
:1049A00090E00196877099278093B003BECFA6E070
:1049B000B0E0EDEDF4E20C94D4300E94F2088C01EA
:1049C00080915C0290915D028017910771F01982CD
:1049D0001A820E94F208BC0149815A8180E090E06D
:1049E00037DF10935D0200935C022696E4E00C949E
:1049F000F030A6E0B0E0EFEFF4E20C94D630909304
:104A0000590280935802811520E2920730F40E94E7
:104A100010112696E2E00C94F23080EF89838A83AD
:104A20000E94F2088160BC0149815A8181E091E0D5
:104A30000FDFEFCFA6E0B0E0E0E2F5E20C94D43077
:104A40008C019093590280935802011580E2180757
:104A5000B0F4802F0E942511C801805E910908974B
:104A600028F063EA71E10115110511F464E971E1BF
:104A7000C8010E94ED032696E4E00C94F03080EF2C
:104A800089838A830E94F2088160BC0149815A812E
:104A900081E090E0DDDEEFCFCF93DF93D82FC92FF9
:104AA000A8DF8D2F9C2FC6DFDF91CF9108950F9344
:104AB0001F93CF93DF938C01862F69E872E00E94E9
:104AC000B317892B91F4C0918902D0918A02209763
:104AD00061F0F8018281833039F4CE01DDDFCE014F
:104AE000DBDFCE01D9DF01C0E0F7DF91CF911F916D
:104AF0000F9108950F931F93CF93DF938C01EB01D8
:104B000069E872E08C2F0E94B317892B09F057C017
:104B1000FE01FF27D80112968C911297E950FE4FA3
:104B20008130A9F415968C9182FD4EC080FF4CC057
:104B300082E0808380918B0290918C020097B9F47F
:104B40008091890290918A020097C9F110C0823049
:104B5000A1F515968C9182FD26C080FD0AC083E0E8
:104B6000808380918D0290918E020097F1F041DF59
:104B700026C084E0808380918F02909190020097FC
:104B8000B1F78091890290918A02009701F184DF48
:104B900080918B0290918C02009749F78091890255
:104BA00090918A02E4CF85E0808380918902909180
:104BB0008A02009721F070DFF1CF86E08083DF91D9
:104BC000CF911F910F91089581E08083B9CF80919B
:104BD0008B0290918C02B8CF0F931F93CF93DF93EA
:104BE0008C01EB0169E872E08C2F0E94B317892BCE
:104BF00071F4DD27C950DE4F8881F80112821882D6
:104C00008330E9F048F4813059F0823081F0DF914F
:104C1000CF911F910F9108958430B1F08530B9F78D
:104C20008091890290918A02009789F306C0809151
:104C30008B0290918C02009799F3FCDEE8CF809173
:104C40008D0290918E02F7CF80918F029091900209
:104C5000009799F72091890230918A0280918B0206
:104C600090918C0221153105F9F2009731F7C901B5
:104C7000E4CFA0E1B0E0EFE3F6E20C94C830FE012F
:104C8000319680E1DF011D928A95E9F707E010E097
:104C900099E9A92E93E0B92E27E6422E512C612CDA
:104CA000712C4F0173016201B1E14B165104610493
:104CB00071041CF080E1C82ED12CA601B501C401FD
:104CC0000E94BE31AC0CBD1C0D2C000CEE08FF0880
:104CD0004C185D086E087F080150104019F7609667
:104CE000E0E10C94E4306FEF85E290E00E94CD317A
:104CF0006FEF86E290E00E94CD316FEF87E290E0A7
:104D00000E94CD3160E088E290E00E94CD310E94A7
:104D1000BE16AFDF66E385E290E00E94CD3165E02C
:104D200086E290E00E94CD3167E287E290E00C9449
:104D3000CD31CDB7DEB7AC970FB6F894DEBF0FBE5E
:104D4000CDBF85B7806885BF85B7806885BF84B7CC
:104D5000877F84BF0FB6F894A89580916000886122
:104D600080936000109260000FBE80E890E00FB664
:104D7000F89480936100909361000FBE81E080936E
:104D800003018DED96E09093C5018093C4010E94CC
:104D9000AF070E9434170E941A0B0E94900B80915B
:104DA000E20084608093E20078948091350281155E
:104DB00099F08091E9001091EC008F701795112700
:104DC0001795182B1092E9008091E80083FD0E944E
:104DD000C40D1F701093E90082E084BD93E095BD7F
:104DE0009AEF97BD80936E00109254021092550274
:104DF00010925602109257020E94A516811101C00E
:104E000072DF8091D80080618093D8002AE12A95D2
:104E1000F1F700C08091D900182F117080FD04C0F7
:104E20000E941A0B109235021093520255985D9809
:104E30008FE891E00197F1F700C0000088274D99B5
:104E400083958093530280930401809152028111D3
:104E50000E94732F809104018091040190E08111E0
:104E600001C095E090930A0285E0891B80930902B6
:104E70000AE411E0D8018D918D018F3F11F00E945D
:104E8000DF06B1E00F341B07A9F70FE411E055E589
:104E9000E52E51E0F52EF80181918F018F3F11F041
:104EA0000E94DF06E016F106B1F78AE0E9E2F2E0DF
:104EB000DF01282F1D922A95E9F7EFEFF1E0DF01DE
:104EC0001D928A95E9F780E090E00E94B931833E17
:104ED0009E4F21F40E94A516811136C063EE7EEF2D
:104EE00080E090E00E94E73160E082E090E00E9484
:104EF000CD3181E08093A70361E083E090E00E94E0
:104F0000CD3160E074E184E090E00E94E7311982E5
:104F1000CE0101960E94DC0CE6DE0E94E20C85E0E8
:104F20000E948A0783E992E00E94DC0C40E050E096
:104F3000BA018FE090E00E94DF3140E050E0BA011A
:104F400083E190E00E94DF3182E090E00E94B13185
:104F500080930D0284E090E00E94B9319093F103B8
:104F60008093F0030E945312EFEFF6E721E0E15047
:104F7000F0402040E1F700C000000E9453128091F1
:104F8000290280FF08C06FEF7FEF80E090E00E9471
:104F9000E7310E94090C83E090E00E94B1310E9449
:104FA0000904259A2D9882E88093800089E18093F6
:104FB00081008FEF9FEF90938700809386000E947F
:104FC000A8150E94A81580915202811101C08ED7A8
:104FD00085E091E090935F0280935E0280913502BC
:104FE000853059F480913502853009F452C00E9411
:104FF0008C0D0E94A8150E9467080E9453120EE0B3
:1050000012E049E2E42E42E0F42ED701F80191913A
:105010008D9128E132E02E173F0709F471C09817EF
:10502000B1F380905202D12CD701CD907D01F801CF
:1050300091908F019C1431F19C24B12CAA24A3944B
:10504000892D8A218115B9F08114A9F0B982DA82FB
:105050000E94F2089C838B83F1E0FD8391E08C2D0C
:105060008A21811101C090E09E8349815A816B8120
:105070007C818D81EDDBB394AA0C26E0B212E0CFE7
:10508000F801C292D3943AE0D312CECF0E94170A0D
:105090003AC080913502843039F180E00E948A075D
:1050A00010920B0288E190E0A0E40FB6F894A89566
:1050B000809360000FBEA093600083B7817F8460FF
:1050C00083BF83B7816083BF7894889583B78E7FD1
:1050D00083BF0FB6F894A895809160008861809393
:1050E0006000109260000FBE0E945312E9E2F2E0ED
:1050F000819181110AC5B2E0E333FB07C9F772CF92
:1051000098138FCF54DC80915202811509F478C036
:1051100000911503109116030115110591F1C0902E
:105120001C02D0901D02E0901E02F0901F020E940F
:105130000B0A6C197D098E099F09C0901802D09046
:105140001902E0901A02F0901B026C157D058E0585
:105150009F05B8F0C8010E9410111092150310921B
:10516000160310921C0210921D0210921E02109241
:105170001F02109218021092190210921A02109235
:105180001B02E0909D03F0909E03E114F10439F1BD
:10519000C0909F03D090A0030E94F2088C010C19CC
:1051A0001D09C7010E94C81780179107C0F42091FC
:1051B0009D0330919E03C9019927287F3327232B14
:1051C00009F02FC134E0880F991F3A95E1F7835E0B
:1051D0009C4FDC0115962C9122FF0E94D2118091E8
:1051E0009402811569F00E94F20820919502309195
:1051F0009602821B930B8F3F9F4710F40E94AD11C4
:1052000086E0E3E8F2E0DE01119601900D928A95C6
:10521000E1F7B0908402D0908502F0908602C090B1
:105220008702E09088021092850210928602109206
:105230008702109288028F2D8D29811509F441C0B3
:1052400000912202109123020E94F2089C01201B6F
:10525000310B90918102911509F452C42531310529
:1052600080F19F3F19F09F5F90938102D11459F014
:105270000E941D0891E01D140CF09FEF899F802D66
:10528000112480938502F11459F00E941D0891E0C9
:105290001F140CF09FEF899F802D112480938602AC
:1052A00080918502811569F010918602111549F0EF
:1052B0000E940F0880938502812F0E940F0880931F
:1052C00086028C2D8E29811509F441C0009120029F
:1052D000109121020E94F2089C01201B310B909139
:1052E0008002911509F407C42135310580F19F3FF3
:1052F00019F09F5F90938002C11459F00E943D08FD
:1053000091E01C140CF09FEF899F802D1124809355
:105310008702E11459F00E943D0891E01E140CF040
:105320009FEF899F802D11248093880280918702AE
:10533000811569F010918802111549F00E940F083B
:1053400080938702812F0E940F08809388028091AA
:1053500084028B1119C080918502811511F08D1185
:1053600013C020918602211511F02F110DC09091CC
:105370008802911511F09E1107C0309187023111FA
:1053800003C0822B892B81110E94270986E0FE0130
:105390003196A3E8B2E001900D928A95E1F70E9460
:1053A000670890912402891721F0809324020E94BB
:1053B0000B0A80913502843009F010CE83E080938F
:1053C000E9008091E80082FF09CE8091E80090E03A
:1053D00085FF05C00E94E90A811531F191E08091B5
:1053E000E8008B778093E800911509F4F7CD0091E0
:1053F0005A0210915B02E9810115110589F1EE3F16
:1054000009F050C08A81833020F08550833008F045
:1054100049C0EA81EE3008F045C0F0E0EA5AFD4CA0
:1054200044C780E090E0D5CE00E210E0FE01319666
:105430007F018091E80085FD0AC08091E8008B77AC
:105440008093E8000E94E90A811599F3C7CF809103
:10545000F100D7018D937D010150104051F7BECF6F
:10546000E43148F4E11549F0E150E33130F4F0E083
:10547000EC59FD4C1AC7EE3F61F28FEF898312C0E1
:105480001A8289E08B830EC08A81823081F083305A
:10549000B1F0813091F70E940B0A0DD76B837C83AA
:1054A0008D839E83CE0101960E94390B97CD88E2B1
:1054B00090E057D71B821C821D828E83F3CF809190
:1054C000330290913402892B69F38AE0E9E2F2E039
:1054D000DE01139601900D928A95E1F7E3CF8A8160
:1054E000823059F66B817C818D819E81E4D688E281
:1054F00090E053D7D7CF4C816B818A810E94CB1526
:105500009827892798279E838D83CCCF2D813E8134
:105510003227232732274C816B818A810E94F80C25
:10552000C1CF0E94BE16BECF8A81893009F0BACFA2
:105530008B81B7E08B9FC00111246FEF70E06CD6B8
:10554000862F0E948A07AECF8A81893029F08A305F
:1055500009F0A8CF1B82A6CF8091930286958695ED
:105560008695EFEF8E9FC001112467E070E054D65E
:105570006B8398CF83E992E00E94DC0C93CF80E2AA
:105580008A8390CF1A8287E67DCF8C818D3108F097
:1055900089CF8A809B80982489249824A12CB12CBF
:1055A0008E010F5F1F4F7801E80EF11C0E151F05CD
:1055B00009F478CF80E0F7E68F169104A104B104D6
:1055C00020F4C40187569C4FCCD6D80114968C93F6
:1055D0000F5F1F4FBFEF8B1A9B0AAB0ABB0AE6CFC8
:1055E0008091330290913402892B09F45BCF8C8136
:1055F0008D3108F057CF882E912CA12CB12CCA8068
:10560000DB80DC24CD24DC24E12CF12C8E010F5F27
:105610001F4F412C512C3201481459046A047B0459
:1056200008F040CFE7E6CE16D104E104F10438F4E7
:10563000D80114966C91C60187569C4FAED6BFEF29
:105640004B1A5B0A6B0A7B0AEFEFCE1ADE0AEE0AF0
:10565000FE0A0F5F1F4FE0CF0CDB24CF86E090CF18
:105660008C818D3108F01ECF882E912CA12CB12C6D
:10567000CA80DB80DC24CD24DC24E12CF12C412CFD
:10568000512C32018E010B5F1F4F481459046A04DC
:105690007B0408F007CF80E0F0EDCF16F2E0DF06E4
:1056A000E104F10418F4C60189965BD6D8018D9304
:1056B0008D01BFEF4B1A5B0A6B0A7B0AEFEFCE1A24
:1056C000DE0AEE0AFE0AE1CF2C81022F10E02D3116
:1056D00008F0E8CE8A819B819827892798272C019A
:1056E000612C712C803DF2E09F0708F0DBCE822E0A
:1056F000912CA12CB12C40ED52E060E070E04419F7
:10570000550966097709421751056105710508F4C5
:10571000C9CE2091330230913402232B09F03EC0D0
:105720001C0129E2220E311C80FBEE24FF24E0F84C
:1057300080FF0BC0889615D69D81892798278927D9
:1057400081159C4711F48FEF8D83D501C401840D21
:10575000951DA61DB71D80FF19C0680181E0C81AFC
:10576000D108DE011596AC0DBD1DBCA7ABA7C101CC
:10577000800F911FF6D5EBA5FCA5908181159C4764
:1057800021F48FEFABA5BCA58C938601FE01319669
:10579000EE0DFF1D2FEFE016F10638F08E010F5FC2
:1057A0001F4FC12CD12C760125C094818581811594
:1057B0009C4711F42483258332E0E30EF11C3296DA
:1057C000EACF80ED481682E058066104710430F497
:1057D000D80114966C91C2018996DFD5BFEFCB1A20
:1057E000DB0AEB0AFB0AEFEF4E1A5E0A6E0A7E0A2C
:1057F0000F5F1F4FC814D904EA04FB0410F352CE04
:105800008091330290913402892B09F44BCECE0162
:1058100001960E94390BFFEF21EE34E0F150204059
:105820003040E1F700C00000B4CB88E0E2E3F1E0F3
:10583000DE01919601900D928A95E1F7FE01329674
:105840008FE1DF011D928A95E9F786E0898388E080
:105850007F96DE0115963ECE88E4898381E08A83B7
:105860001B821C821FCE8B819C81092E000CAA0BEF
:10587000BB0B25E0880F991FAA1FBB1F2A95D1F7E4
:10588000AC01BD01405E5F4F6F4F7F4F4817590716
:105890006A077B0708F406CE8834E1E09E07A1057D
:1058A000B10508F0FFCD4934F1E05F0761057105EE
:1058B00020F048E451E060E070E0481B590BBC0167
:1058C00064537A4FCE01019616D5ECCD4AE150E0F3
:1058D0006FEF70E0CE0107962DD58091330289835A
:1058E0000A831B821C821D8281E0E7CD81E090E06B
:1058F00090935B0280935A0282E390E09093280297
:10590000809327020E94F20890932602809325023A
:10591000C9CD0115110571F1D0902902E090250241
:10592000F09026020E94F2088E199F098536910593
:1059300040F1D1FE26C0D0FE24C00E94F208909310
:1059400026028093250280912702909128020197D8
:105950009093280280932702892B61F410925B02B6
:1059600010925A0281E090E09093340280933302C7
:1059700000E010E08091330289830A83809127023E
:1059800081CD82E390E09093280280932702F2CFAA
:10599000109234021092330285CD40E250E06FEF56
:1059A00070E0CE010196C6D47DCD8B81823009F4A2
:1059B00050C078F4811136C0FE0132968EE1DF01CD
:1059C0001D928A95E9F788E089838B8383E088A319
:1059D00069CD853009F472C0863009F063CD1C8131
:1059E0008AE0FE013596DE01919601900D928A952E
:1059F000E1F78BA19CA10E94A2079CA38BA38FEF30
:105A0000183060F4FAE01F9FB0011124675B7C4FEF
:105A10004AE050E0CE018196DED480E089830E9486
:105A2000341740CD8C819AE0F92E8E010F5D1F4F07
:105A3000F8012F2D11922A95E9F7B8010E94B317AA
:105A40008983F801DE01129601900D92FA94E1F734
:105A500029CD1C818AE0FE013596DE0191960190E8
:105A60000D928A95E1F789A19AA10E94A2079AA3B3
:105A700089A38BA19CA10E94A2079CA38BA38DA1AB
:105A80009EA10E94A2079EA38DA38FA198A50E940C
:105A9000A20798A78FA38FEF183060F43AE0139F06
:105AA000B001112467507D4F4AE050E0CE0181964D
:105AB00092D480E089830E94AF07F4CC2C816AE005
:105AC000CE018196DC01E62F1D92EA95E9F7283098
:105AD00080F4629FB0011124675B7C4F4AE050E084
:105AE00030D480E089838AE0FE01B196DE0112960F
:105AF000F1CC8FEFF7CF2B30310508F0FACB27CC64
:105B00002B30310508F0AFCBDCCB80910C02811536
:105B100009F468CAE0E1E9BDF2E1F9BD09B400FEAB
:105B2000FDCF8091D8008F7D8093D8008091E000D8
:105B300082608093E0008091E00081FDFCCF0E94B4
:105B40008C0D50CA1F921FB61F9211248F939F93E2
:105B5000AF93BF9380910B02811113C08091EE012E
:105B60009091EF01A091F001B091F1014196A11D3A
:105B7000B11D8093EE019093EF01A093F001B093DB
:105B8000F101BF91AF919F918F911F901FBE1F9008
:105B9000189578941F921FB61F9211248F939F938C
:105BA000AF93BF938091EE019091EF01A091F0012E
:105BB000B091F1010196A11DB11D8093EE0190936A
:105BC000EF01A093F001B093F101BF91AF919F91CC
:105BD0008F911F901FBE1F9018951F920F920FB6A6
:105BE0000F9211242F933F934F935F936F937F9363
:105BF0008F939F93AF93BF93EF93FF938091E100B7
:105C000082FF09C08091E20082FF05C08091E1001F
:105C10008B7F8093E1008091DA0080FF24C0809127
:105C2000D80080FF20C08091DA008E7F8093DA0058
:105C30008091D90080FFA9C080E189BD82E189BD42
:105C400009B400FEFDCF81E0809335028091DD0133
:105C5000811109C00E941A0B0E94900B8091E200F2
:105C600084608093E2008091E10080FF1AC08091FF
:105C7000E20080FF16C08091E2008E7F8093E200F8
:105C80008091E20080618093E2008091D800806280
:105C90008093D80019BC85E08093350283E080931F
:105CA00003018091E10084FF2FC08091E20084FF16
:105CB0002BC080E189BD82E189BD09B400FEFDCF22
:105CC0008091D8008F7D8093D8008091E1008F7EF5
:105CD0008093E1008091E2008F7E8093E2008091CA
:105CE000E20081608093E2008091DC01811509F47B
:105CF00052C084E08093350280913502843009F0EF
:105D000052C082E0809303018091E10083FF2CC0A8
:105D10008091E20083FF28C08091E100877F80931B
:105D2000E10082E0809335021092DC018091E10075
:105D30008E7F8093E1008091E2008E7F8093E2006D
:105D40008091E20080618093E20042E060E080E0C8
:105D50000E94600B8091F00088608093F00081E0E9
:105D60008093030180930201FF91EF91BF91AF9166
:105D70009F918F917F916F915F914F913F912F9163
:105D80000F900FBE0F901F90189519BC10923502FE
:105D90001092DD0168CF8091E30087FF02C083E0AD
:105DA000A9CF81E0A7CF81E0ADCF1F920F920FB6B0
:105DB0000F921124EF92FF920F931F932F933F9313
:105DC0004F935F936F937F938F939F93AF93BF9303
:105DD000CF93EF93FF9309EE10E0F8018081C0911B
:105DE000EC008F70C795CC27C795C82B108280EF29
:105DF000E82EF12CF7018081877F808378940E94C0
:105E0000C40DF8011082F701808188608083CF7013
:105E1000F801C083FF91EF91CF91BF91AF919F9116
:105E20008F917F916F915F914F913F912F911F9132
:105E30000F91FF90EF900F900FBE0F901F9018954D
:105E40008EE1489B02C08A95E1F7489BFECF0895FA
:105E5000589880E28A95F1F7589A0895FC012BE052
:105E60002A95F1F728E090E080E031E040E14A95A2
:105E7000F1F7880F489B02C08160932742E04A9562
:105E8000F1F7000040E14A95F1F72A9579F720E112
:105E90002A95F1F729B132E03A95F1F7000040E197
:105EA0004A95F1F7217092272081920F90830895EF
:105EB000A1E0B0E0EDE5FFE275C119828C017C0143
:105EC000E60EF11CBDDFCE010196C8DFF80181931B
:105ED0008F01EE15FF05B1F781E09981911180E006
:105EE0002196E6E07BC1509A589A08955098589AA6
:105EF000E89AE9E6F0E080818C7F80830895615024
:105F0000770B91E001C0990F6A95EAF7692F90E04D
:105F100021E0611108C0911599F0589A80E28A95A4
:105F2000F1F758980895362F3823311539F0589ADB
:105F3000922730E23A95F1F76695EBCF5898F9CF72
:105F40005898ECCFFF920F931F93CF93DF93EC0100
:105F50008C01060F111DF9907BDF68E08F2DCFDFDC
:105F6000C017D107C1F7CDB7DEB7E5E038C11F9242
:105F70000F920FB60F9211240F931F932F933F93FD
:105F80004F935F936F937F938F939F93AF93BF9341
:105F9000EF93FF93CF93DF930F92CDB7DEB71982C4
:105FA0004FDFCE0101965ADF082F0695069506951C
:105FB000982F92959570202F2570920F292F23707E
:105FC00096959695920F982797708981892B8115C0
:105FD00009F058C0053008F055C080E18A95F1F706
:105FE000589A509A82E08A95F1F700C0589888E054
:105FF000089F80011124D801AF5EBE4F1696ED9127
:10600000FC9117973097A9F0609155017091560156
:1060100014962D913C911597260F371F11968D914F
:106020009C911297680F791F13964C9113978C913E
:106030000995F801EF5EFE4F6381611549F02091EB
:1060400055013091560184819581820F931F7ADF2B
:10605000FFDE80E18A95F1F758985098589A80E1D0
:106060008A95F1F7F801EF5EFE4F6081611549F006
:10607000209155013091560181819281820F931FA9
:1060800017DFDEDE0F90DF91CF91FF91EF91BF918F
:10609000AF919F918F917F916F915F914F913F91C0
:1060A0002F911F910F910F900FBE0F901F90189579
:1060B0000F931F93CF93DF938C0105970CF05EC075
:1060C000F894509A589885E08A95F1F70000C02F0F
:1060D000C695C570802F8570C80F8C2F8370C695AC
:1060E000C69593E0000F111F9A95E1F7C80FC801FC
:1060F0008C2BEC01ADDE00C068E08C2F00DF90E15E
:106100009A95F1F75098589A489B31C087E090E0F3
:1061100048992FC0F801EF5EFE4F6381611559F079
:10612000209155013091560184819581820F931FF2
:10613000BFDE811501F184DE80E28A95F1F758987F
:10614000509A90E19A95F1F7F801EF5EFE4F608169
:10615000611549F02091550130915601818192815C
:10616000820F931FEFDE74DE789481E008C000C0D8
:10617000CBCF019749F4509A589A789480E0DF91F8
:10618000CF911F910F91089500C0C2CF2F923F92DF
:106190004F925F926F927F928F929F92AF92BF9237
:1061A000CF92DF92EF92FF920F931F93CF93DF93E3
:1061B000CDB7DEB7CA1BDB0B0FB6F894DEBF0FBE40
:1061C000CDBF09942A88398848885F846E847D848D
:1061D0008C849B84AA84B984C884DF80EE80FD808F
:1061E0000C811B81AA81B981CE0FD11D0FB6F89405
:1061F000DEBF0FBECDBFED010895DB018F939F93EE
:1062000070D0BF91AF91A29F800D911DA39F900D63
:10621000B29F900D11240895AA1BBB1B51E107C02A
:10622000AA1FBB1FA617B70710F0A61BB70B881F26
:10623000991F5A95A9F780959095BC01CD010895B5
:1062400097FB072E16F4009406D077FD08D0E4DF04
:1062500007FC05D03EF4909581959F4F0895709569
:1062600061957F4F0895A1E21A2EAA1BBB1BFD0169
:106270000DC0AA1FBB1FEE1FFF1FA217B307E40725
:10628000F50720F0A21BB30BE40BF50B661F771F7D
:10629000881F991F1A9469F760957095809590955D
:1062A0009B01AC01BD01CF010895EE0FFF1F0590CA
:1062B000F491E02D09946927962769277827872785
:1062C00078270895A29FB001B39FC001A39F700DCE
:1062D000811D1124911DB29F700D811D1124911DEE
:1062E0000895F0DFA59F900DB49F900DA49F800DA1
:1062F000911D11240895FB01DC0102C005900D924F
:1063000041505040D8F70895FB01DC0104C08D9145
:106310000190801921F441505040C8F7881B990B17
:106320000895FB01DC0102C001900D9241505040E4
:10633000D8F70895DC0101C06D9341505040E0F75B
:106340000895DC01CB01FC01F999FECF06C0F2BD36
:10635000E1BDF89A319600B40D9241505040B8F723
:106360000895F999FECF92BD81BDF89A992780B51D
:106370000895A8E1B0E042E050E0E5CFDC01A40FD1
:10638000B51F4150504040F0CB01840F951F2E9116
:1063900005D041505040D8F70895262FF999FECFE7
:1063A00092BD81BDF89A019700B4021639F01FBA68
:1063B00020BD0FB6F894FA9AF99A0FBE0895039685
:1063C000272FECDFEADF252FE9DF242FE7CF019627
:1063D000272FE4DFE2CFDC01CB0102C02D9105D0F5
:1063E00041505040D8F70895262FF999FECF1FBA93
:1063F00092BD81BD20BD0FB6F894FA9AF99A0FBEEE
:1064000001960895F894FFCF5C0961096309680952
:106410007809780978097809780978097809780974
:106420006A096E097109760986098C099009A10E1D
:10643000C70ECD0EC70ECD0E1F0F400FCD0E46104E
:1064400053106B1ED31E731E3D1E411E771E451E2C
:106450007B1E871E511ECC1E551E8B1E591E8F1E65
:10646000B41E5D1E931EBB1E631E991EA11E491EF7
:106470007F1E4D1E831E671E9D1EAB1EC41ECA1EA0
:10648000371E6F1EDA1E091E0F1EFC1D031E151E71
:106490001B1E211E232023205A205A200B21262197
:1064A0007E207E202B219F21B021B021152C2C2C69
:1064B000332C522A522A662C762C892CC82CCD2CAF
:1064C000522A522A522AD52C402A442A6F2A7B2A41
:1064D000862A912A942AA42ABA2A3D2A002CBF2A65
:0E64E000C22AC52AF02A2C2B2E2B302B642B1F
:1064EE000000010001EF086F0C700A850C8A0C6623
:1064FE000C0000000100000000000000050100007B
:10650E00000406000000000000010A000000000068
:10651E000001BBBBAD3D7081F6410044227B4901B9
:10652E002701AC004F0268028802F0F597F6F7F1EA
:10653E00F4379293943E02E200E900EA00B500B609
:10654E0000B700CD008301CC008A01920194012195
:10655E0002230224022502260227022A02B300B4D5
:10656E00006F0070009F01CB019F02A002E200E9C4
:10657E0000EA00B500B600B700CD008301CC008A5A
:10658E0001920194012102230224022502260227F0
:10659E00022A02B300B4006F0070009F01CB019F6E
:0465AE0002A0020045
:00000001FF
